:1078000011241FBECFEFDAE0DEBFCDBF0BC14101B7
:1078100042144505560455026403740300001E9586
:1078200087020110030000C18081C106C0FF0A0069
:107830000CA10185037508150026FF00954009017C
:107840008102954009029102C0040309041A033021
:1078500000300030003000300030003000300031A7
:1078600000370030003100380341007200640075B9
:107870000069006E006F0020004C0065006F006E14
:10788000006100720064006F00200062006F006FF2
:107890000074006C006F00610064006500720018E5
:1078A00003410072006400750069006E006F0020E3
:1078B000004C004C00430012010002020000404155
:1078C0002334000001000203011201000200000045
:1078D0004041233400000100020301090264000357
:1078E00001008032080B00020202010009040000BE
:1078F0000102020000052400100105240101010419
:107900002402020524060001070581031000400936
:10791000040100020A0000000705020240000007FF
:107920000583024000000904020001030000000971
:107930002101010001221E000705840340004000D0
:1079400020918A0130918B012C5F3F4F30938B0146
:1079500020938A01C901892F99278695982F803411
:1079600018F08FE7891B982F990F921710F44798FA
:107970000895479A08955D9A289A81E08093E000DF
:107980001092E200EE27FF270994089528E088E18D
:1079900090E00FB6F894A895809360000FBE2093F6
:1079A0006000FFCF0F931F93CF93DF93982FEB01CE
:1079B000042F10E088E76030780730F411E083E0AE
:1079C000FB0180935700E895892F68E071E0402F14
:1079D00006D1112311F107B600FCFDCF402F4695CB
:1079E000FE01A8E0B1E020E031E009C08D919D9159
:1079F0000C0130935700E895112432962F5F24171D
:107A0000A8F385E0FE0180935700E89507B600FCD7
:107A1000FDCF81E180935700E895DF91CF911F91D1
:107A20000F91089584B794B7977F94BF98E10FB6EC
:107A3000F89490936000109260000FBE5D9A289AAF
:107A4000479883FF08C0E0E0F0E0859194918F5F54
:107A50009F4F09F090DF3F9A209A559A90E89093B3
:107A600061001092610081E885BF95BF9FD084E1DD
:107A70008093880180E180938901E0E0F0E08591C6
:107A800094918F5F9F4F19F081E080938F01EE24D6
:107A9000FF24BB24B39454EFC52E51E0D52E1FD242
:107AA000082F8EE098E7FC012491319602964491CC
:107AB000201711F02223B9F7109291011092900132
:107AC00082E068E071E08BD0013479F460910801C4
:107AD0006058633028F0683111F064E001C063E061
:107AE000C62FD0E0CF5DD7480EC0063571F4809127
:107AF0000801803311F011E022C080910A01C82FE3
:107B0000D0E0C25ED74811E022C0053721F413E06F
:107B1000CEE1D8E71CC0053539F4E0900801F090BB
:107B20000901EE0CFF1C0AC0043631F482E0B701F3
:107B30004091090137DF02C0043721F010E0C5E2AF
:107B4000D8E705C010910901E701E10EF11CC7D18A
:107B50008097B1F483E068E871E041E050E059D0EB
:107B6000112329F0412F50E083E8BE0152D083E475
:107B700069E871E041E050E04CD0013509F08FCF69
:107B8000D0929101C0929001B0928F01EE24FF2417
:107B900086CFFC01289884E680938D0104C08091F3
:107BA000F100819361506623D1F7089510929101FD
:107BB0001092900110928E0110928F0181E08093BB
:107BC000D70080EA8093D80082E189BD09B400FE25
:107BD000FDCF80E98093D8001092E0000895FB016A
:107BE0008093E90024E69BE611C08091E80085FFC0
:107BF000FCCF289820938D018091F1008193809192
:107C0000E80085FD02C09093E8004150442369F7E5
:107C10000895982FFB01282F207287708093E90028
:107C200064E63AE317C08091E80085FFFCCF97FF38
:107C300002C0849101C080813196211180E05D985D
:107C400060938C018093F1008091E80085FD02C073
:107C50003093E800415050408FEF4F3F580719F7DD
:107C600096FF03C08AE38093E80008958091930112
:107C7000813299F45D9884E680938C0120E030E0B5
:107C800003C080818093F100F901E050FF4F2F5F26
:107C90003F4F28303105A9F714C0803261F480913C
:107CA000E80082FFFCCF80E091E067E072DF8BEFBD
:107CB0008093E80006C0823221F480919401809381
:107CC000070181E0089520919501223291F1213040
:107CD00081F48091980190919901089711F4209373
:107CE0009A0180919A01882309F059C029EC38E75C
:107CF00058C0223029F484E690E02BED38E71DC00F
:107D0000233009F04AC080919401882319F429E4B2
:107D100038E747C0823019F427E638E742C083309D
:107D200019F42DE438E73DC08130B9F52FE938E783
:107D300038C082E090E02BE238E740919801509102
:107D40009901BC014817590708F4BA0190918C01B8
:107D500040E050E0AEEF8091E8008570E1F3809163
:107D6000E80082FD16C0F901E40FF51F4F5F5F4F79
:107D7000E4915D98E093F100842F8F7311F4A09348
:107D8000E80094E64617570730F390938C0181E0A2
:107D9000089590938C0180E0089580E0089527EB8A
:107DA00038E7F901849190E0C8CF1092E900809102
:107DB000E80083FF61C082E991E068E0EADE82EFDB
:107DC0008093E8008091920187FF05C08091E800D0
:107DD00080FFFCCF03C08EEF8093E8008091930179
:107DE000853051F48091E80080FFFCCF80919401B0
:107DF00080688093E30039C08930E1F48091940178
:107E000080938E01E7E2F8E791E031E026E390937A
:107E1000E9003093EB0084918093EC002093ED0017
:107E20009F5F3196953099F78EE78093EA00109224
:107E3000EA001BC0883049F490918E015D9884E679
:107E400080938C019093F10010C0882339F45D98E1
:107E500084E680938C011092F10007C0863011F403
:107E600032DF01C003DF882321F08EEF8093E8002A
:107E7000089581E28093EB0008958091E1001092D3
:107E8000E100282F83FF0CC01092E90081E080936D
:107E9000EB001092EC0082E38093ED0010928E01D3
:107EA00022FF1CC080918C01882331F08150809387
:107EB0008C01882309F45D9A80918D01882331F02B
:107EC000815080938D01882309F4289A80918F0135
:107ED000882321F4109291011092900108951F932C
:107EE000CF93DF9312E0C0E9D1E05FDFC6DF1093EC
:107EF000E9008091E80085FF13C0289884E680930C
:107F00008D019091F1008091E80085FD03C08BE622
:107F10008093E800892F90E0DF91CF911F91089521
:107F2000809190019091910101979093910180939C
:107F300090018091900190919101892B09F426DDA7
:0A7F4000CE010197F1F7FCDCD0CF71
:087F4A0000E10000000000004E
:040000030000780081
:00000001FF
